:030000000219FDE5
:03000B000200AA46
:03002B0002015F70
:03005B000202E7B7
:030073000202CDB9
:1000800002030406080C10182030406080040608A3
:100090000C10182030406080A0C000070F1F3F0DDB
:1000A0000D04050D050205030302C2AFC0D0C0E078
:1000B000206217E5256002E473E525F4F58A758B67
:1000C00000D262D0E0D0D0D2AF3285268AC262E5BB
:1000D00026F4602F758B00D0E0D0D0D297D295D285
:1000E00093D2AF32D297D295D293206E0C2066096C
:1000F0007405D5E0FDE57E4290758B00D0E0D0D050
:10010000D2AF32758A00C28DD26201F901B930686E
:1001100005206602C29701B9306805206602C293C5
:1001200001B9306805206602C29501B9C2963068EF
:100130000A206607740FD5E0FDC29701B9C292305C
:10014000680A206607740FD5E0FDC29301B9C29416
:1001500030680A206607740FD5E0FDC29501B9C268
:10016000AFC2AD53E6EFC0D0C0E0D2D3D2AFC2CE63
:10017000E52A6007207449152A21C07800790020FB
:10018000742EE580307E01F430E50278FF53DACF3B
:10019000207E0343DA20307E0343DA10C2D8C271D6
:1001A000E580307E01F430E50279FFC3E89970CB39
:1001B000306103752A18207403752A18885FD2707D
:1001C00020740DE52B6004152B21D043DA01C2D831
:1001D000207002412EA85F206102C270207436791F
:1001E00082B70431C3E894F0400374F0F8E8C454D3
:1001F0000F28F87984B703024115C313C31387216D
:10020000200802C313200A06C3C898F8411528F82D
:10021000500374FFF88822E52D54066011E533C3BE
:1002200013C31324062522F52250037522FF78827A
:10023000B6044E852224A824C3E52495644002A870
:1002400064C3E895664002A8668825E569700241A6
:100250007FC3E8AA699A5003E8FAE4F9EAC333FBDA
:10026000E56BF45B29400D256AF8E56A6002156AC2
:10027000400B417F0AC3E56A9A5002056A78FF88FD
:1002800026C3E52594404002D26420CF0AD0E0D0B6
:10029000D043E610D2AD32C2CF053A7801E52A60EC
:1002A00005307402152AC3E55F94014005756200AC
:1002B00041C3756300756C00E5622401F56250036B
:1002C0007562FFD0E0D0D043E610D2AD32C2AFC0ED
:1002D000D053E67FC2607591008556948557957519
:1002E0009104D0D0D2AF32C2AF53E6EFC2ADC0D08E
:1002F000C0E0C0F0D2D3D2AFA8FBA9FCC2D8307105
:1003000002614E53DACF207E0343DA10307E03437E
:10031000DA20D271E580307E01F420E50261258883
:10032000278928A17553DACF207E0343DA20307E57
:100330000343DA10C2D8C271307402A1617800E5BB
:1003400080307E01F430E502A161885FA14953DA73
:10035000CF207E0343DA20307E0343DA10C27120BF
:100360006102812753DACF207E0343DA10307E0307
:1003700043DA20C2D8D271885A895BC3E89558F80D
:10038000E99559F97B007E087A00C3E8948CE994DA
:10039000005005755E008119882178A2E6A82160C9
:1003A00055C3E894C8E994005008E4D2E4FB7A0A03
:1003B00061F4C3E89468E994015008E4D2E3FB7A5D
:1003C0000F61F4C3E894D0E994025008E4D2E2FB50
:1003D0007A1E61F4C3E894A0E994055008E4D2E1E0
:1003E000FB7A3C61F4C3E89498E994085008E4D29D
:1003F000E0FB7A787E00C3E8955CFCE9955DFD3012
:10040000E70AECF42401FCEDF43400FD755E00C352
:10041000EC9AED9E5003755E01885C895D855A58A3
:10042000855B597802A149C3E89527F8E99528F931
:10043000307C02A12D307B02A12D307A02A1262032
:100440007502814AE9FDE8FC8169E9C313F9E81303
:10045000F8307902A126E9C313F9E813F8307802DD
:10046000A126E9C313FDE813FC206126C3EC941C0C
:0E047000ED940240028180ED7018C3EC94C838
:10047E0050120529C3E529940A5002A161755F0047
:10048E00D270A161E529600215297888E6F9740019
:10049E00207F087896B90302789EE624FAFEE434AB
:1004AE0000FFC3EC9EFCED9FFD9208B90310A2085D
:1004BE005007207609D27681CC307602C276A20819
:1004CE005016B9030DECF42401FCEDF43400FD02DA
:1004DE0004E678007900A12DB90315EC33FCED3359
:1004EE00FDC3EC940AFCED9400FD50047C007D00ED
:1004FE00C3EC94FFED9400400678FF7900A12DEC3B
:10050E008575F0A4C5F0A2F733F879004003020513
:10051E004978FF7900020549E9C313F9E813F83069
:10052E007C0EE9600278FFC3E81338F8E43400F972
:10053E00C3E894FFE99400400278FF885FD27020F0
:10054E006102A161741FF4552F4BF52FC274EB702D
:10055E0002D274752A18307403752A0A306102A10A
:10056E007520740353DAFE207403752B06D0F0D079
:10057E00E0D0D0D2AD43E6103279010205A5790361
:10058E000205A5790A0205A5791E0205A579640260
:10059E0005A579C80205A57817E4D5E0FDD8FAD9E6
:1005AE00F6227A147B780205CC7A107B8C0205CC6D
:1005BE007A0D7BB40205CC7A0B7BC80205CC79028E
:1005CE00B27DE4C292D5E0FDC293D5E0FDD293D5C3
:1005DE00E0FDD292D5E0FDC297E576D5E0FDD2974B
:1005EE007496D5E0FDD9D9EAF8D5E0FDD8FBDBCE7F
:1005FE00C29222C37C007D0075F00005F0EA33FA4A
:10060E00EB33FB50F6EB13FBEA13FAC3E9FFE8FEFC
:10061E00E89AF8E99BF95004EFF9EEF8B3EC33FCE5
:10062E00ED33FDD5F0DFEDF9ECF822E889F08A2004
:10063E00D2D4F8A9F07B0030F70B7BFFF42401F83D
:10064E00E9F43400F9E88520F0A4ADF0F8E985204E
:10065E00F0A4AFF0FEED2EF974003FFA7C04C3EA6D
:10066E0013FAE913F9E813F8DCF48BF030F70AE823
:10067E00F42401F8E9F43400F9E889F0C2D4F8A9B9
:10068E00F0227882B604030206EBC3E55F940140C4
:10069E00030206B5852224E4F545F546F547F548EF
:1006AE00F549C26D0206EB7882E6FCD26DE522F5C5
:1006BE0023783879C7AA40AB41C3EB13FBEA13FA90
:1006CE00EC146013C3EB13FBEA13FAEC141460077B
:1006DE00C3EB13FBEA13FAD1018845894622C3E521
:1006EE00459523F8E5469400F9500CC3E89480E94B
:1006FE0094FF401602071CC3E8947FE99400500350
:10070E0002071C787F790002071C788079FF884ADF
:10071E00894B22E54A2547F8E54B3548F9854B20AC
:10072E00E4300701F43549FA30E709C3EA94F040A2
:10073E001502075AC3EA940F500302075A78FF793D
:10074E00FF7A0F02075A780079007AF0C3E52495F4
:10075E0064500AC374019524500B020778E54B20B0
:10076E00E70E020778E54B30E706884789488A4945
:10077E002278A4E6FAC3E54A33F8E54B33F9D139CA
:10078E00E930E70BC3E89480E994FF4013E1B2C36C
:10079E00E8947FE994005002E1B2787F7900E1B2EB
:1007AE00788079FFE820E715C3E52398F84009C360
:1007BE00E8940140030207D978010207D9E8F4242E
:1007CE00012523F840030207D978FF884C2278A52B
:1007DE00E6FAA848A949D139E930E70CC3E89401F3
:1007EE00E994FF401602080DC3E894FFE994005007
:1007FE000302080D78FF790002080D780179FFE9F0
:10080E0020E715C3E54C98F84009C3E8940140036E
:10081E000208347801020834E8F42401254CF8402B
:10082E000302083478FF88242278FFC26420693DD1
:10083E00206A12D264C3E541940A4009C3E52594A7
:10084E00405002C26479A1E76023E541601F74FF46
:10085E008541F0848539F0306A0375F005A4F8C53A
:0F086E00F0600278FFC3E895675002A8678866BC
:10087D0022C3E5409440E5419401E566500314011F
:10088D008F046002F566220208972275E89022789F
:10089D0083E6FFE5E820ECF7A8BDA9BE0573C3E527
:1008AD007394084052757300E9FA79A0E76044EA41
:1008BD007007E574601B0208D2C3E895746010E5FB
:1008CD00745006600C140208DE0460F90208DEE5BF
:1008DD0074F574C3946D401B7564C0C394044013C8
:1008ED00756480C39404400B756440C39404400345
:1008FD0075640075BB0822E5642410500274FFF581
:10090D00647982B70402212BC3A864E524985002B0
:10091D00A824C3E895664002A86688258826E57355
:10092D00B4070375BB1022743279A687F0A4C5F005
:10093D00A2F733F8C3E895644002A864882288249E
:10094D00882588268867227540007541F022C2AF40
:10095D0075C820A8CCA9CDAA3A30CF010A75C824F4
:10096D00D2AFAB3BAC3C883B893CC3E89BF8E99CE0
:10097D00206908F9306702417021CDAD3D8A3DF9FE
:10098D00EA9DFA600478FF79FFAE3EAF3F8B3E8C57
:10099D003FC3EC9FFCC3E99CF542A83BA93CC3E8CF
:1009AD009EF8E99FF9C3E54113FBE54013FAE82AE8
:1009BD00F540E93BF54150067540FF7541FF411784
:1009CD00AA40AB41AC40AD417E047F02C3EB940421
:1009DD0040021E1FC3EB940840021E1FC3ED13FD02
:1009ED00EC13FCDEF7C3EA9CFAEB9DFBEF6009C349
:1009FD00E913F9E813F8DFF7EA28FAEB39FB8A4037
:100A0D008B4150067BFF8B408B41C3EB9402500210
:100A1D00D2673069047F0341427892E6FFC3E53720
:100A2D00948240110FC3E53794A040010FC3EF949A
:100A3D000640027F057E06E541C4540FF9E541C429
:100A4D0054F0F8E540C4540F28F8C3E89EFAE99431
:100A5D0000FB4009C3EA9402EB940050047A02E4CF
:100A6D00FB41BCAA40AB41EBC4FEEAC4540F4EFCA3
:100A7D00C3EA9CFAEB9400FBC3E813C313F8EA280E
:100A8D00FAEB3400FB8A408B41C3EB94024002C267
:100A9D00677806EBC4FE7B00EAC4540F4EFAC3EA36
:100AAD0098FA4005C3940250027A027892E6FF301C
:100ABD00600241BC855256855357D26043E680C3D0
:100ACD00E49AF8E49BF93067026156E8FAE9FBD342
:100ADD00E913FDE813FC88528953C3EF9403603882
:100AED00EF20E00DE82CF8E93DF9ECFAEDFB020BF7
:100AFD0011E828F8E939F9C3E82402F8E93400F9D6
:100B0D007AFE7BFFC3EF9403400E8A548B55884EBB
:100B1D00894F8C508D51618A885489558A4E8B4FDF
:100B2D008C508D51306920C3E53394034019E54253
:100B3D00A2E713F8E555F4240138400B20E70875BA
:100B4D0054FFF42401F555618AE8FAD3E813FC88C3
:100B5D0052C3EF94036020EF20E007E82CF8ECFA85
:100B6D006176E8282402F87AFEC3EF940340088AE0
:100B7D0054884E8C50618A88548A4E8C50E56BC3D4
:100B8D00335002646BF56B3060026194753402D2A0
:100B9D006043E680E52D54066026A840A941C3E9CF
:100BAD0013F9E813F8C2AF53E67F759100C3E498CB
:100BBD00F594E499F595759104D26043E680D2AF32
:100BCD0022D265754400752000306B0375204002FC
:100BDD000BEDD265754400752040306B0375200018
:100BED00D2AF7801206722E52D54066002C265C39D
:100BFD00E541940540137802940540087803940567
:100C0D0040027806306902780A206019E5446015C3
:100C1D0030690AC3E53394034003D53406D2AFD20D
:100C2D006C81BE719CD2AF0000C2AF206726E5413A
:100C3D00C3FB940F40027B0FEB240530730123306F
:100C4D006A02742820620123F93069027982E58BEA
:100C5D00C39940B50544E59B5440B5200281A830A9
:0F0C6D00690A08C3E8940A40010881162065024D
:100C7C0061EDC26553E67F75910030671075940085
:100C8C007595FE759104D26043E68061EDAE40AF80
:100C9C0041C3E49EF594E49FF595818FC3E53394AD
:100CAC0002500261ED30650261EDD80281BC811603
:100CBC00C26C53E67F75910085549485559575915A
:100CCC0004854E56854F57D26043E680D2AFE52D52
:100CDC0054066008206A020533020CF8306C0D20B3
:100CEC006B0A2065071581158102155E227800308C
:100CFC0064053065027801E53775F007A4F9E5F075
:100D0C0028F5F0E9A2F013A2F113A2F213F537C300
:100D1C0094785003753778C3E53795384008D26618
:100D2C00D297D295D293306002A13285505685511C
:100D3C0057D26043E68022207D11C2AF754302C2B8
:100D4C0092D296D2AF759F13020F12C2AF754302A7
:100D5C00C292D294D2AF759F13020F1230724320FD
:100D6C007D20C2AF75430390013D757E04D295C2C0
:100D7C0094306204C293A186D292D2AF759F1002B6
:100D8C000F12C2AF75430390013D757E04D297C21A
:100D9C0096306204C293A1A6D292D2AF759F110273
:100DAC000F12207D17C2AF754303900118D29530F6
:100DBC006202C293D2AF759F10020F12C2AF75437D
:100DCC0003900118D297306202C293D2AF759F1173
:100DDC00020F12207D11C2AF754304C296D294D279
:100DEC00AF759F11020F12C2AF754304C294D29615
:100DFC00D2AF759F10020F12307243207D20C2AF0C
:100E0C0075430590012C757E40D293C292306204DA
:100E1C00C297C122D296D2AF759F13020F12C2AFE6
:100E2C0075430590014E757E10D293C292306204C8
:100E3C00C295C142D294D2AF759F13020F12207D7E
:100E4C0017C2AF75430590010ED293306202C29760
:100E5C00D2AF759F13020F12C2AF754305900122DA
:100E6C00D2933062EBC295D2AF759F13020F122052
:100E7C007D11C2AF754306C294D292D2AF759F104A
:100E8C00020F12C2AF754306C296D292D2AF759FB3
:100E9C0011020F12307242207D20C2AF75430190B7
:100EAC00014E757E10D297C296306204C295C1BEB7
:100EBC00D294D2AF759F11020F12C2AF754301903D
:100ECC00012C757E40D295C294306204C297C1DE6B
:100EDC00D296D2AF759F10E112207D16C2AF75432A
:100EEC0001900122D297306202C295D2AF759F1148
:100EFC00E112C2AF75430190010ED295306202C26D
:100F0C0097D2AF759F10C2662290010C757E00D2ED
:100F1C0097D295D293C296C294C292C26222788022
:100F2C0076090876090876040876FF0876030876B1
:100F3C00FF08760B087601087601087601788C7626
:100F4C00010876FF0876FF0876FF0876FF0876FF23
:100F5C000876030876FF0876FF0876FF08762508E2
:100F6C0076D00876280876500876040876FF08763E
:100F7C000208760008767A0876FF08760108760172
:100F8C00087600087603227887E6FFC2727888E636
:100F9C00C394036008C27DE630E102D27DC27E7844
:100FAC0089E630E102D27EC3EF94026008758E01AF
:100FBC00D273020FC6758E00C273227880E614902D
:100FCC0000809378A4F67881E6149000809378A53D
:100FDC00F67886E61490008D9378A6F6789CE675E4
:100FEC0038FF75390CB402067538A075390AB4038C
:100FFC000675388275390578A3E61490009A93F536
:10100C0069120F1522227896E6FA7897E6FB788813
:10101C00E6B40305C3EB940EFB307F047A007BFF30
:10102C00C3EB9AFCC3948250027C827575000575E3
:10103C00EC8575F0A4C3E5F0947D40F222D27F11CB
:10104C00121205967A007B007C1012058CE55F2A43
:10105C00FA74003BFBDCF37C04C3EB13FBEA13FADE
:0D106C00DCF7FEC27F111222E5EF20E60343
:101079007520000520903FFFE520146006901DFFB4
:101089001460009304600375EF1253D9BF7581C0D2
:1010990043FF8012058775EF0243B203E5B32404C9
:1010A90020E70DF521E5E320E0068521B343E301BF
:1010B900120F157580FF75A40075F1B275D4DF752F
:1010C90090A975A5FC75F2FE75D50175A60175E2A5
:1010D90041E4F8F6D8FD756B01120F2A1215A078B4
:1010E900988676753001C2AF1205A01205B01205B7
:1010F900961205B71205961205BE120596C2AF786B
:10110900FA79FA308507D9FBD8F7021C00120F9338
:10111900120FC71111111278988676120F1575885A
:101129005075891275C82475910475D84075A8221F
:1011390075B80275E690759B80759D0075D10E7521
:10114900BC5875BB0875BA1175E880120587D2AF0E
:1011590012089453DACF207E0343DA20307E03430A
:10116900DA1043DA01C2D8C2711205A0D2617B0339
:101179007A0CE55E70077A0CDB03021106120596FC
:10118900207003021106C270E55FC3940240E1E5D5
:101199002F541F856160F561B560D5DAD5C26153F9
:1011A900DACF207E0343DA20307E0343DA10C2D837
:1011B900C27178A2E67008D274E52F54E0F52FC207
:1011C9007575290012059B307409C3E529940A40F5
:1011D90002D27512058C78023074027800C3E55F7B
:1011E9009840F0C2AF1205B01205B01205B0D2AFE7
:1011F9001205A0754D007888E6B4030241DD120599
:101209008C788CE6C3940150030212DDE530C39457
:101219000150030212DD207435C3E55F94FF5003CA
:101229000212DDC2AF1205C5D2AF12059BC3E55F3D
:10123900940150EFC2AF1205B01205911205B0D258
:10124900AF12059BC3E55F94FF40E90217487F028F
:10125900D27F111212059BC2AFC27F1112AE5FC3BA
:10126900E55F947FD2AF4076120587C2AF1205C5FC
:10127900D2AFDFDC1149C3EE94057897F61205A0C9
:101289001215E21216CB7F0AD27F111212059BC2E8
:10129900AFC27F1112AE5FC3E55F947FD2AF50E654
:1012A900120587C2AF1205B01205911205B0D2AF6F
:1012B900DFD61149EE24057896F61205A01215E23B
:1012C9001216FA12059B1112C3E55F94FF500241F1
:1012D9001F021748C3E55F954D4003855F4D120511
:1012E9009B78017988E7B403027805C3E55F9840E4
:1012F9000221FFC2AF1205C51205C51205C5D2AF3D
:101309001205A0753000E4F531F5320531E531F407
:1013190070390532789AE6781914601278321460B7
:101329000D787D14600878FA146003753200C3E5FE
:101339003298401715327531B478998676C2AF1252
:1013490005C5D2AF7898867612059B120591E52AD4
:101359007005307402210678012074027806C3E50D
:101369005F9840A77888E6C39403600312059BE55C
:101379002A7003021106C2AF120F15E4F522F523F4
:10138900F524F525F526F56AD2AF7885E6C333F558
:1013990068E4F545F546F547F548F549F573F52C43
:1013A900F52DF53775730875BB1012058712089866
:1013B900E5E820ECFBA8BDA9BEE97001F888741224
:1013C900089C75730875BB107887E6FE7602120FC4
:1013D900937887EEF6C2AF7564FF120934852264EB
:1013E900852265852266D2AF75220175240175258E
:1013F9000175260185636C756D017888E6B403076C
:10140900C27D307602D27DD268D269753300120E60
:101419007B120EA012095412095B12095412095BBE
:1014290012095402143CC2AF120F93D2AF75730064
:1014390075BB08120BDF120690120CF9120D43123C
:10144900095B120BCE306D031206EC2067031208FC
:101459003730670312087E120CF9120D6812095B06
:0F146900120BDF306D03120721120CF9120DDF89
:1014780012095B120BCE306D0312077F120CF912A2
:101488000E0412095B120BDF306D031207DC120C1D
:10149800F9120E7B12095B120898120BCE120CF986
:1014A800120EA012089C12095B306935206B328538
:1014B800676485676585636C756D0179187A0CC3F7
:1014C800E53399400FC269D26A8A358567648567B2
:1014D800660214E9C3E55F9401400302143C021557
:1014E80066306A1B206B18E535147004C26A812FB8
:1014F800F535C3E55F9401400302143C0215667597
:101508003600C3E56278FA985054307404E52A60CE
:101518004D7888E6B40317207D05207607A136307C
:101528007602A136206B07D26B856764817B78F0E1
:10153800306B058567647820C3E541985002813C8B
:10154800306B1BC26BC27D307602D27DD26A753594
:1015580012856764813C0536E55F6002A1697536CE
:1015680000C2AF120F157887E6FE7602120F937845
:1015780087EEF6E4F522F523F524F525F526F5683A
:10158800C268D2AF120587120F15307409C3E53649
:10159800940540022106610F901A0D782012162436
:1015A800E520B4550CA3121624E520B4AA030215AD
:1015B800C2120F2A1215E20215E1901A0378807BF5
:1015C8000A121624A308DBF9901A0F788C7B1812DC
:1015D8001624A308DBF9901A2722C2AF1216631249
:1015E800163D901A00740E121629A37404121629B7
:1015F800A37414121629901A0378807B0A121628ED
:10160800A308DBF9901A0F788C7B18121628A30808
:10161800DBF9121676121654901A2722E493F62252
:10162800E6438F01538FFD75EF0275B7A575B7F1C6
:10163800F0538FFE22438F02438F0175EF0275B777
:10164800A575B7F1901A0DF0538FFC22901A0D74FE
:1016580055D129901A0E74AAD129227A3079D078D6
:1016680020901A40D124E520F709A3DAF7227A302E
:1016780079D0901A40E7D12909A3DAF922AB77A8E3
:1016880078BB01027980BB02027981BB03027982AF
:10169800BB04027984BB05027986BB06027992BB3A
:1016A80007027987BB080279A3BB0902799CBB0AA8
:1016B800027988BB0B027989E8F7227C051205A01C
:1016C800DCFB22C2AF1205B01205B71205BE120527
:1016D800C51205911205B01205B71205BE1205C54F
:1016E8001205911205B01205B71205BE1205C5D232
:1016F800AF22C2AF1205C51205BE1205B71205B05A
:101708001205911205C51205BE1205B71205B012D1
:1017180005911205C51205BE1205B71205B0D2AF64
:1017280022AE77AF78C2AF1205B01205B01205B07D
:10173800120591DEF21205C5120591DFF8D2AF222B
:10174800D1CBD1C3D1C3757701757801757900F113
:10175800297C05AD5F1205A0C3ED955F70F5C3E563
:101768005F9401400AC3E55F94FF4032021784D1B9
:1017780085B1E2D1CBC2AF75EF12D1C3DCD5057903
:10178800C3E5799403500280C6D1C30578E5771480
:1017980090009F93F808C3E57898500280AED1C3B3
:1017A800D1C30577C3E577940C5002809C120F2AA9
:0917B800B1E2C2AF75EF12D1C31A
:0319FD0002107461
:101A00000E0414090904FF03FF0B01010155AA018B
:101A1000FFFFFFFFFF03FFFFFF25D0285004FF0259
:081A2000007AFF01010003FF41
:101A4000235475726E696779364123202020202047
:101A500023424C48454C4923463333302320202031
:101A60002020202020202020202020202020202076
:101C0000C2AFC2D353D9BF7581C043B20343FF8073
:101C1000752438752503B1C975EF0275E24043F1AB
:101C20002053A4DF75D400D2857DFA780379E67C51
:101C300010752200752300901DD67B0675249875BB
:101C400025013085028142208508D8FBD9F9DCF7CF
:101C500081B4308508D8FBD9F9DCF781B4B189E4C7
:101C600093A3C39A6004DDC381B4DBDBB17B600264
:101C7000812B7B08E493FAA3B15CDBF87A30B15C8A
:101C8000752200752300B17BEAFCEBFDC3ED94FEE9
:101C9000400EB17B8A278B28ED30E0048A828B834B
:101CA000B17B7AC270D8C3ED94FE601350CEBD00F4
:101CB00025EC60097520007521FF0200008100A855
:101CC00027A9280809D804D90281D3B17FEA89AAB3
:101CD000F281C50D81A0C3ED94035049EDA2E092BD
:101CE000007AC5C3E5829400E583941C50902000DF
:101CF00010438F02438F0175B7A575B7F1F030001F
:101D00001FA827A9280809438F01538FFDD804D99C
:101D100002A12089AAE275B7A575B7F1F0A3A10DBC
:101D2000538FFC817C7AC1BD030CE493A3FAB140CC
:101D3000DCF8B138817C817EAA22AB23B15CEBFA5E
:101D4000EA6222752608C3E52313F523E52213F57D
:101D50002250066323A0632201D526EAB1C9B1C986
:101D600075260AEAF4200102D285300102C285B14B
:101D7000C9C3134002C201D526EB22B17FEAFB2082
:101D80008502A17F308502A184752608AE24AF2587
:101D9000C3EF13FFEE13FEB1CDB1C9C3EA13308513
:101DA000024480FA30E703632201C3E52313F523DD
:101DB000E52213F52250066323A0632201D526D91C
:101DC000E52265236523F52222AE24AF250E0FDE22
:101DD000FEDFFCD20122424C48656C693437316326
:041DE000F3300601D5
:00000001FF
